:10713600420520000042040B00004204060000C184
:0571460014C113C11289
:0A935A00C213C214E490040AF022CA
:10903A00E4900520F0A3F090040BF0A3F0A3F090C5
:10904A000406F0A3F090040104F0A3E4F0900409EC
:02905A00F02202
:0693730012935A02903A29
:1091E100E4F5848FC343C30175C04475CF8EC2C3F8
:0991F10043E60290040804F02298
:10501B00E4F58420C7FDC2C2129373E4900408F038
:01502B002262
:0B931800E4F584D2C290040804F022A7
:0D92F100AE071291E1900405EEF0029373B8
:108FF000E4900678F0A3F0301302FF222014FDD293
:1090000013900403E4F0A37410F090050EEFF0E465
:04901000A3F07F0149
:019014002239
:108E8E0030130A900403E07002A3E070037F002207
:108E9E00900404E024FFF0900403E034FFF090050A
:108EAE000FE0FE04F074102EF582E43405F583EF26
:048EBE00F07F01221E
:0B932300301307C213D2141292432231
:10924300900678E584F0E4F58420C7FDC2C4D2C556
:06925300900678E0F584AE
:0192590022F2
:108713008B2F8A308931900408E07002FF22E53202
:108723006005D3941040037F0022128FF0EF604363
:10873300E4900677F0900677E0FFC39532501FABC5
:108743002FAA30A9318F8275830012624BFF128EDC
:108753008EEF7002FF22900677E004F080D7E4905A
:10876300040AF0129323E53370032014FD90040AE6
:03877300E0FF2202
:038776007FFF2260
:0673C1008B2C8A2D892EA1
:1073C700E490066CF0D3900521E09400900520E04E
:1073D7006480948050037F002253E6FD900406E00A
:1073E700FEA3E0240DF58274043EF583E090066C5D
:1073F700F0900406E475F0011262ACFEE4B5F00B00
:10740700EEB40107E4900406F0A3F0900402E00450
:10741700F07006900401E004F0E490066DF0900629
:107427006DE0FFC39D505F90066CE0FEEFC39E507A
:1074370055900406E0FEA3E0240DF58274043EF5A2
:1074470083E0FFAB2CAA2DA92E90066DE0F582757F
:107457008300EF12628A900406E475F0011262ACB1
:10746700FEE4B5F00BEEB40107E4900406F0A3F0D8
:10747700900402E004F07006900401E004F0900626
:107487006DE004F0809890066CE0FFA3E0C39F5086
:1074970030900406E475F0011262ACFAE4B5F00B23
:1074A700EAB40107E4900406F0A3F0900402E004B4
:1074B700F07006900401E004F090066DE004F0809F
:1074C700C5900521E024FFF0900520E034FFF0434C
:1074D700E602EFC39D500790066CE0FF8002AF0500
:0174E7002282
:10921300D3900521E09400900520E0648094804081
:08922300047F0180027F00229C
:03501800026FD64E
:106FD600C0E0C0F0C083C082C0D075D000C000C081
:036FE60006C007DB
:106FE900C20AAFC1EF12639E701F08701F10702F85
:106FF90018703420704128706E3070793870816053
:10700900707C68708170707C7870898070899071EB
:1070190002A00000711090050EE0F5C2C2C59005EE
:107029000DE4F002711290050F802890040A74FD96
:10703900F0D2C4D2C502711290050FE0FF90050D80
:10704900E0C39F5014E0FF04F074102FF582E4347C
:1070590005F583E0F5C2027112D2C490040AE4F086
:10706900C214027112D2C590040A74FEF0027112A0
:10707900027107D212027112900400E4F002711237
:10708900900400E07020E5C2F0E0FFC3900402E044
:107099009F7480F8900401E0648098500312903A3C
:1070A900900400E004F0900402E024FFF090040151
:1070B900E034FFF090040BE0FEA3E0240DF58274A8
:1070C900043EF583E5C2F090040BE475F001126209
:1070D900ACFEE4B5F00BEEB4010790040BE4F0A3A9
:1070E900F0900400E014F07020900521E004F070A5
:1070F90018900520E004F0801030120DC21290059E
:107109000DE4F0D2C58002D20A300A0EC2C6D2C638
:0C711900C2C5C2C4D2C2C20AC214C2C3A2
:10712500D007D006D000D0D0D082D083D0F0D0E028
:017135003227
:05937900A2C7E433FF70
:01937E0022CC
:088C5F008B298A2A892B8D2C38
:108C6700E4900675F0AB29AA2AA92B852C32852D0D
:108C770033E4FF128713900676EFF0BFFF0D9006DF
:108C870075E0FF04F0EFC3940340DA900676E0FF47
:028C97007E005D
:018C990022B8
:068FCA008B298A2A892B85
:108FD0007E007F007D101263C4AB29AA2AA92B7DD5
:0F8FE000101273C190066BEFF07002FF227F0139
:018FEF00225F
:10889B0090066B7422F0A3EFF0A37413F012623204
:1088AB0090066EF090000112624B90066FF09000F4
:1088BB000212624B900670F090000312624B90060E
:1088CB0071F090000412624B900672F0900005124A
:1088DB00624B900673F090000612624B900674F098
:0E88EB007B017A06796BE4F52D7D0A028C5F25
:1090C00090066B7422F0A3EFF0A37403F0A374FF77
:0F90D000F07B017A06796BE4F52D7D04028C5F4D
:1090DF0090066B7422F0A3EFF0A3741CF0A374FF3F
:0F90EF00F07B017A06796BE4F52D7D04028C5F2E
:10913A00E490066BF0A3EFF0A3740AF0A3EFF07BC0
:0D914A00017A06796BE4F52D7D04028C5F3F
:06937F00C2C253E6FD220C
:10727F00AB37AA38A939853D45853E46853C47AD94
:05728F0036AC35AF3400
:0C7294008F3F8C408D418B428A4389441F
:1072A0009006727403F0A374E8F0AD84E4F58420D2
:1072B000C7FDC2C4D2C2D2C5E4900671F0F57630E3
:1072C000C3FDAFC1EF24F8602324F8601F24F860E9
:1072D0003024F8603824F8603924F87003027370A1
:1072E00024F87003027375243802737A900671E0F3
:1072F000700BE53F25E044A0F5C27403F0C2C580E1
:107300007CE540F5C29006717405F08070757603D7
:10731000806B900671E0FFB40509E541F5C2740683
:10732000F0805AEF64067035E5477010AB420544B3
:10733000E544AA437002054314F98006AB42AA4310
:10734000A944126232F5C2E546154670021545E5BC
:1073500046454570289006717407F08020900671AC
:10736000E0B40707D2C47409F08012757605800D69
:10737000757604800875760680037576019006712F
:10738000E0B40904C2C38033E576B4031D900672ED
:1073900074FFF5F01262AC45F0600FD2C4D2C5D2D2
:1073A000C2C2C3E4F576900671F0E5766008C2C506
:1073B000D2C4C2C38005C2C30272BF20C7FD8D8480
:0173C00022AA
:0C7732008F348C358D368B378A388939BE
:10773E00753C03753DE885843EE4F58420C7FDD293
:10774E00C2C2C4D2C5E4FFF57630C3FDAEC1EE129F
:10775E00639E77850077880877881077AA1877B2A6
:10776E002077B72877CD3077D23877D74077E35068
:10777E00780C5800007785027812C2C5EF700CE5C0
:10778E003425E044A0F5C27F03807CEF640170775E
:10779E00E53425E044A1F5C27F04806BE535F5C2E2
:1077AE007F058063757603805EBF0508E536F5C2FA
:1077BE007F068053BF0606D2C57F01804A801175B1
:1077CE0076048043757606803EBF04047F028037C0
:1077DE007576058032AB370539E539AA3870020562
:1077EE003814F9E5C2126278E53B153B7002153A82
:1077FE00E53B453A7004C2C2800D7F028009D2C4B7
:10780E007F098003757601BF0904C2C3802FE57618
:10781E00B40319E53D153D7002153C14453C600C52
:10782E00D2C4D2C5D2C2C2C3E4F576FFE5766008F3
:10783E00C2C5D2C4C2C38005C2C302775720C7FDDA
:03784E00853E84F0
:017851002214
:0C7E53008F348C358D368B378A38893996
:107E5F007E00E536543FFF543F6050C374409FFD92
:107E6F00E49EFCC3E53B9DE53A9C5008853A3D8571
:107E7F003B3E80048C3D8D3E12727FE57660037F22
:107E8F000222E53E2536F536E53D3535F535E53C3F
:107E9F00700CE53E2539F539E53D3538F538C3E544
:107EAF003B953EF53BE53A953DF53A853A3D853BA9
:107EBF003ED3E53E9400E53D9400405AE53E9440A4
:107ECF00E53D9400501112727FE57660037F022228
:107EDF00E4F53DF53E80DAAB37AA38A93975450090
:107EEF0075464012728BE57660037F022274C025BF
:107EFF003EF53E74FF353DF53D74402536F536E4CD
:107F0F003535F535E53C70A974402539F539E4353B
:087F1F0038F538027EC07F0036
:017F27002237
:1092AE00753A00753B01127732E57660037F012235
:0392BE007F00220C
:10925A008B757B007A007975753A00753B01E4F5E8
:05926A003C127E5322BE
:1092C10085323A85333B127732E57660037F01229E
:0392D1007F0022F9
:0D92FE0085323A85333BE4F53C127E532265
:0893640033302E3220202000DE
:10714B00C110C18F4106B4004106B3004106B00027
:10715B004106B1014106B5004106B2004106B60039
:04716B00C10DC10E83
:10926F0030B30930B2037F28227F292230B2037F27
:05927F002A227F2B22D2
:108DB700900635E0FEA3E0FF90066BEEF0A3EFF020
:108DC70090063BE0FDA3E090066DCDF0A3EDF0EF3C
:108DD7004E7012D3E094FF90066DE0940040069029
:058DE70006B37401F069
:018DEC002264
:10409A0075FFDE75FFADE4F5E6F5E7128AD920A6CD
:1040AA00047F0180027F009006B4EFF0128A8E121C
:1040BA004D8F1289F412926F9006B7EFF0C2A79053
:1040CA000680E025E025E024CBF582E43405F5837B
:1040DA00A3E0FAA3E0FFEA4480FAA9079005C5E441
:1040EA00F0A3EAF0A3E9F0900681E025E025E024B8
:1040FA00EBF582E43405F583A3E0FAA3E0FFEA4492
:10410A0080FAA9079005C8E4F0A3EAF0A3E9F0E46D
:10411A00FF12932E9006A4E0FF900697E0FD128509
:10412A00B9900698E0FF1290A0900686E0FF128FE1
:10413A007A90069AE0FF128F27900686E0FF128F88
:10414A007A900699E0FF128EC212934F124D8F1287
:02415A007D7472
:10415C00C207E4F526C210301E08200705128DB7E1
:10416C00D2079006B6E0600BA3E0FF1290C0E4907B
:10417C0006B6F0201B030245F2C21B12842C7F01F1
:0F418C00129174EF60419006B1E0602AE4F525CE
:10419B0074FFF527F528E5281528AE27700215279B
:0841AB00D39400EE940050EEE5
:1041B3000525E525B480E1127852E49006B1F0902C
:1041C3000686E02402FF128F7A7F01128E23D20E1D
:1041D3007F04128B64EF601B90069AE004F0C39493
:1041E300034002E4F090069AE0FF900560F0128F1E
:1041F30027D2107F05128B64EF601B900699E004B1
:10420300F0C394034002E4F0900699E0FF90056147
:10421300F0128EC2D2107F07128B64EF601B9006E0
:1042230086E004F0C394084002E4F0900686E0FFC1
:1042330090055FF0128F7AD2101292D48F249006D9
:10424300A4E06524600DE524F0900697E0FD128557
:10425300B9D21012926F9006B7EFF0E4FF12917487
:10426300EF60279006B2E06021E4FF128E239006F0
:10427300B0E070149006B7E0FF7BFF7A9379641285
:10428300889B9006B07401F0D20DE4FF128B64EFAB
:1042930060419006B2E0601FE49006B0F0300D0478
:1042A300C20D802C900697E06401F0FD9006A4E017
:1042B300FF1285B902415CE4900697F09006A4E0F2
:1042C300FFE4FD1285B9E4FF12930BE49006B5F009
:1042D300127D74128395EF6002D2107F01128B64FA
:1042E300EF6022300E04C20E801B900698E004F0AB
:1042F300C394044002E4F0900698E0FF90055EF05A
:104303001290A0D210128E597D157F011263F07D99
:104313000E7F0A1263F07D067F081263F07D037F30
:10432300091263F07D17E4FF1263F07D167F02121A
:1043330063F07D147F031263F0E4FD7F041263F0E6
:104343007D017F051263F07D057F061263F07D0218
:104353007F071263F07D0D7F0B1263F07B017A06FA
:10436300794F128FCAEF70030245E9900651E012AC
:10437300639E43F90444460543B71443941643A389
:104383001743C01A43E21B43ED1D43F31E000044D1
:10439300999006977401F09006A4E0FF7D01800CCC
:1043A300E4900697F09006A4E0FFE4FD1285B9D2ED
:1043B300100244999006B27401F00244997B017A89
:1043C30006794F90065FEBF0A3EAF0A3E9F01262DF
:1043D30032FE9006B7E0FF6E6003024499800590B9
:1043E30006B7E0FF1290DF02449912936C024499DE
:1043F3001293850244997B017A06794F900662EB0A
:10440300F0A3EAF0A3E9F090000312624BFF9006D9
:10441300B7E06F6003024499900697E060709006DE
:1044230062EBF0A3EAF0A3E9F090000512624BFF00
:1044330090000612624BFD90000412624BFB128443
:10444300B4804B7B017A06794F900662EBF0A3EAC6
:10445300F0A3E9F090000312624BFF9006B7E06F00
:104463007034900697E06026900662EBF0A3EAF0C2
:10447300A3E9F090000512624BFF90000612624B15
:10448300FD90000412624BFB1282EA75260190062E
:10449300B7E0FF12913A900697E0700302459890B7
:1044A3000651E014603C24FA605B1470030245502B
:1044B30024F97003024584240D60030245981250C9
:1044C3001B7B017A06794F90065FEBF0A3EAF0A31A
:1044D300E9F090000312624BFF12930B127D7402FA
:1044E300457F12501B7B017A06794F90065FEBF0F4
:1044F300A3EAF0A3E9F090000312624B900522F0C7
:10450300752601807712501B7B017A06794F90063E
:1045130065EBF0A3EAF0A3E9F090000312624BFF0E
:1045230090000412624BFD90000512624BFBC00326
:10453300900665E0FBA3E0FAA3E0F990000612629F
:104543004BF52CD0031280C3752601802F12501B0C
:104553007B017A06794F900665EBF0A3EAF0A3E9B5
:10456300F090000312624BFF90000412624BFD9027
:10457300000512624BFB12684B75260112931880DB
:10458300147B017A06794F900668EBF0A3EAF0A357
:10459300E9F0127B91E5266401600302435F900515
:1045A30022E0FF12932E9006A4E0FF900697E0FD11
:1045B3001285B9900698E0FF1290A0900686E0FF5E
:1045C300128F7A90069AE0FF128F27900686E0FFFB
:1045D300128F7A900699E0FF128EC212934F124DFA
:1045E3008FD20F02435F301006127D74128DED20BF
:0A45F3000F0302415C127D74C20F39
:0345FD0002415C1C
:0A716F0041056500C115410522002D
:06938500E4900565F022F2
:07936C009005657401F02279
:1087790090055EE0900698F090055FE0900686F01F
:10878900900560E090069AF0900561E0900699F0F6
:10879900900562E0900696F0900563E0900681F0FE
:1087A900900564E0900680F0E4FFEF25E02444F5AD
:1087B90082E43405F583E0FCA3E0FDEF25E024A87D
:1087C900F582E43405F583ECF0A3EDF00FBF0DDA83
:0187D900227D
:1087DA00900698E090055EF0900686E090055FF0BE
:1087EA0090069AE0900560F0900699E0900561F095
:1087FA00900696E0900562F0900681E0900563F09D
:10880A00900680E0900564F0E4FFEF25E024A8F5E7
:10881A0082E43405F583E0FCA3E0FDEF25E024447F
:10882A00F582E43405F583ECF0A3EDF00FBF0DDA21
:01883A00221B
:10895200900698E090055EF0900686E090055FF044
:1089620090069AE0900560F0900699E0900561F01B
:10897200900696E0900562F0900681E0900563F023
:10898200900680E0900564F0E4FFEF25E02444F5D2
:1089920082E43405F583747FF0A374FFF00FBF0DFA
:0189A200E9EB
:0189A30022B1
:10785200A2AF9208C2AF900643E0FCA3E0FDECC4E5
:10786200F854F0C868FAEDC4540F48FBECC313FE99
:10787200ED132BFDEE3AFC900643E01313543F7ECA
:10788200002DFFEE3C900566F0A3EFF0900641E07C
:10789200FCA3E0FDECC4F854F0C868FAEDC4540F40
:1078A20048FBECC313FEED132BFDEE3AFC900641B0
:1078B200E01313543F7E002DFFEE3C900568F0A3C9
:1078C200EFF0900627E0FFA3E090056ECFF0A3EF64
:1078D200F0900633E0FEA3E07802CEC313CE13D8B5
:1078E200F9FF900572EEF0A3EFF090062FE0FEA3F1
:1078F200E07802CEC313CE13D8F9FF900570EEF0F4
:10790200A3EFF090063FE0FEA3E0FFC3E49FFF7405
:10791200809EFEEF7803CEA2E713CE13D8F8FF9035
:10792200056AEEF0A3EFF090063DE0FEA3E0FFC390
:10793200E49FFF74809EFEEF7803CEA2E713CE137E
:10794200D8F8FF90056CEEF0A3EFF01293917ED081
:107952007F007B017A05796675360075370E128CC9
:087962009A129190A20892AF65
:01796A0022FA
:10823C00E4F52EF52FF5301293917ED07F0F7B0055
:10824C007A00792F753600753701128C9A7ED07FA3
:10825C000E7B007A007930753600753701128C9AD6
:10826C00129190128952E4900566F0A3F0A3F0A34A
:10827C00F090056EF0A3F0900572F0A3F0900570ED
:10828C00F0A3F090056A7480F0A3E4F0A37480F07E
:10829C00A3E4F01293917ED07F007B017A0579667E
:1082AC0075360075370E128C9A129190129391E4D8
:1082BC00F52D75F021E52DA42400F582E5F034C0F0
:1082CC00AF82FE7B017A0579447536007537211231
:0E82DC008C9A052DE52DC3941E40D70291907B
:108A8E0090D00FE493F4600790D00EE4936005123B
:048A9E00823C803165
:108AA2007AD07900892C8A2B752AFF752900E52C4A
:108AB200F52CE52BF52BE4F52AF5297B017A0579CE
:108AC20066AF2CAE2BAD2AAC29F53475350E128B60
:018AD2002182
:068AD300E4900522F022F0
:108DED002015309006B2E06013900697E060249055
:108DFD000565E0701E9006B604F080179006B574F8
:108E0D0001F0900697F09006A4E0FF7D011285B960
:068E1D00127D74D2152243
:108F5100900522E0FFC3941E501EEF75F021A4245A
:108F610000F974C035F0FA7BFF78447C057D017E01
:098F7100007F2112620CC21522DE
:108EF500900522E0C3941E5028129391900522E01C
:108F050075F021A42400F582E5F034C0AF82FE7B24
:108F1500017A057944753600753721128C9A1291BC
:028F2500902298
:06938B00128EF5C215224E
:0D930B00AE071287DA900522EEF002938B78
:0B932E00900522EFF0128F51028779AA
:0480C3008D2A8B2B4C
:1080C700052C90066DEFF0A3E52BF090066DE0FF11
:1080D700D3952A400302816E75F021EFA42400F5A1
:1080E70082E5F034C0AF8290066FF0A3EFF0900600
:1080F7006EE075F021A42400F582E5F034C0AF826C
:10810700900671F0A3EFF0E490066BF0A3F09006F1
:1081170071E475F0011262C2AFF0FE90066FE0FCE9
:10812700A3E0F5828C83E493FD12853A900670E014
:1081370004F0700690066FE004F090066CE004F01F
:10814700700690066BE004F0C390066CE0942190F3
:10815700066BE0940040B712919090066DE004F032
:10816700A3E004F00280D2900522E0FFE52BD39F25
:0B8177005009E52CC39F400312932E1B
:0181820022DA
:06684B008F298D2A8B2B22
:1068510090066FE529F0A3E52BF090066FE0D39544
:106861002A40030269BBA3E075F021A42400F5824C
:10687100E5F034C0AF8290066BF0A3EFF0E4900630
:1068810071F0A3F0900671E0FEA3E0FFC39421EE46
:106891009400503890066BE0FCA3E0F5828C83E411
:1068A10093FD74232FF582E43405F583EDF0900612
:1068B1006CE004F0700690066BE004F0900672E064
:1068C10004F070C0900671E004F080B890066FE0AB
:1068D10075F021A42400F582E5F034C0AF82900662
:1068E1006DF0A3EFF0900670E075F021A42400F59F
:1068F10082E5F034C0AF8290066BF0A3EFF0E49034
:106901000671F0A3F090066BE475F0011262C2AF5C
:10691100F0FE90066DE0FCA3E0F5828C83E493FD2C
:1069210012853A90066EE004F0700690066DE00460
:10693100F0900672E004F07006900671E004F0C376
:10694100900672E09421900671E0940040B79006A1
:106951006FE075F021A42400F582E5F034C0AF8228
:1069610090066DF0A3EFF0E4900671F0A3F09006AD
:1069710071E0FCA3E0FDC39421EC9400502C90063F
:106981006DE475F0011262C2AFF0FE74232DF58241
:10699100E43405F583E0FD12853A900672E004F0D7
:1069A10070CC900671E004F080C412919090066F53
:1069B100E004F0A3E004F002685B900522E0FFE54B
:1069C1002BD39F501FE529FDE52AC39DFDE49400CB
:1069D100FCE52B7A002DFDEA3CFCC3ED9F7480F8A9
:1069E1006C985011900522E0FFE529D39F500EE5E8
:0D69F1002AC39F4008900522E0FF12932E5C
:0169FE002276
:0682EA008F298D2A8B2B69
:1082F000A2AFE43390066BF0C2AF12937FE52AFF82
:10830000E529900670CFF0A3EFF0E490066CF090B2
:108310000670E0FCA3E0FD7B017A0579237532004D
:10832000753321AF2B1292C1900671E02421F09099
:108330000670E03400F090066CE075F021A4240093
:10834000F974C035F0FAA374FFF0A3EAF0A3E9F0E2
:1083500012939190066DA3E0FAA3E0AE02FF7B01B9
:108360007A057923753600753721128C9A1291900F
:1083700090066CE004F0E0C3941E4093900522E068
:10838000FF12932E9006B7E0FF1292F190066BE079
:0483900024FF92AF85
:0183940022C6
:0684B4008F298D2A8B2B9D
:1084BA00A2AFE43390066BF0C2AF12937FE52AFFB6
:1084CA00E52990066DCFF0A3EFF0E490066CF090EA
:1084DA00066CE0FFC3941E504675F021EFA42400F9
:1084EA00F582E5F034C0AF82FE90066FF0A3EFF09C
:1084FA0090066DE0FCA3E0FDAA06A9077BFF753292
:10850A0000753321AF2B1292FE90066EE02421F003
:10851A0090066DE03400F090066CE004F080B090B4
:0F852A0006B7E0FF1292F190066BE024FF92AFCC
:01853900221F
:0E92E3000001000200040008001000200040FE
:10717900025D0032410697004106980041068600EB
:1071890041069A0041069900410696004106810090
:107199004106800041068F0041069000410691009A
:1071A90044068700000000440682000000004406EF
:1071B900920000000044068B0000000001650001F8
:0271C90074014F
:106CFB009005C2A3E0FF30E00F90064BE0FBA3E052
:106D0B009005A8CBF0A3EBF09005A9E02400F55675
:106D1B009005A8E03480F555EF30E50F90061FE0A5
:106D2B00FFA3E09005B2CFF0A3EFF09005B2E0FE29
:106D3B00A3E07802CEC313CE13D8F9F5548E53903B
:106D4B000680E0C39405500E900697E06020E55E48
:106D5B006432455D601890056AE0FEA3E0FFC3E472
:106D6B009FF552E49EF551E4F553F55480189006C7
:106D7B003FE06480FEA3E0FF90056BE02FF552909F
:106D8B00056AE03EF551900697E0600AE55E6432D5
:106D9B00455D60028049900643E0C4F854F0C86832
:106DAB00FCA3E0C4540F48FD900643E0C313FEA3BD
:106DBB00E0132DFDEE3CFC900643E01313543F7E95
:106DCB00002DFDEE3CFC30E7047C7F7DFF900566DB
:106DDB00E0FEA3E0FFC3ED9FFDEC9EFC30E703E478
:106DEB00FCFD75C30E8551C28552C1E553C313FE1D
:106DFB00E554138E92F5918555C28556C18C928DB3
:106E0B009175C27F75C1FF856692856791C281C2FC
:106E1B0081C281ACCFADCE900686E030E03075C339
:106E2B000E75C27F75C1FF8C928D918570C2857175
:106E3B00C1E55BC4F854F0C868FEE55CC4540F4868
:106E4B008E92F591C281C281C281ACCFADCEC3EC23
:0D6E5B00648094805003E4FCFD8C6A8D6B14
:016E68002207
:1074E800AB6BAA6A75C3038AC28BC175920075918A
:1074F80008C281C281859651859552E55264074537
:10750800517068F554755340EA540FFCEB54F0750C
:10751800C3038CC2F5C1759208759100C281C281FE
:10752800AC96AD95743C2DF58274603CF583E4937C
:107538007A0075C3018AC2F5C1759200759140C27F
:1075480081C281AA94AB93EB4254EA42537A377BC7
:107558000075C3018553C28554C18A928B91C2813B
:10756800C281AA96AB958A638B6422E4F554E552EE
:1075780025E0FFE55133FE74E32FF58274923EF562
:1075880083740193F553EA540FFCEB54F075C3036D
:107598008CC2F5C1759208759100C281C281AC9602
:1075A800AD95743C2DF58274603CF583E4937A00C4
:1075B80075C3018AC2F5C1E55225E0FFE55133FEE6
:1075C80074E32FF58274923EF583E493FE7401937D
:1075D8008E92F591C281C281AA94AB93EB4254EA90
:1075E80042537A377B0075C3018553C28554C18ADB
:1075F800928B91C281C281AA96AB95EAA2E713FA4F
:06760800EB138A63F56438
:01760E002259
:104F6A009005C2E0FCA3E0FDEC30E30F900637E0C9
:104F7A00FFA3E09005BECFF0A3EFF09005BEE0F5E9
:104F8A0051A3E0F55290062FE0FEA3E07802CEC3CB
:104F9A0013CE13D8F9FF900570E0FAA3E0FBC3EF34
:104FAA009BF554EE9AF553EC30E20F900639E0FF88
:104FBA00A3E09005BCCFF0A3EFF09005BCE0F55557
:104FCA00A3E0F55675C30EE42552FFE5513480F58A
:104FDA00C28FC185539285549175C27F75C1FFE511
:104FEA0055C313FEE556138E92F591C281C281C252
:104FFA0081AFCEAECFC3EE648094805003E4FEFF4F
:04500A008E5B8F5CCE
:01500E00227F
:10667F00900681E0C39405501890063DE06480FEBB
:10668F00A3E0FF90056DE02FFF90056CE03EFE80CC
:10669F000F90056CE0FEA3E0FFC3E49FFFE49EFEB6
:1066AF008E518F529005C2E0FCA3E0FD30E40F90B5
:1066BF00061DE0FFA3E09005B0CFF0A3EFF090052B
:1066CF00B0E0FEA3E07802CEC313CE13D8F9F55491
:1066DF008E53ED30E20F900649E0FFA3E09005AC3A
:1066EF00CFF0A3EFF09005ADE02400F5569005AC88
:1066FF00E03480F555900641E0FCA3E0FDECC4F8D2
:10670F0054F0C868FAEDC4540F48FBECC313FEED08
:10671F00132BFDEE3AFC900641E01313543F7E001D
:10672F002DFFEE3CFE90067EF0A3EFF0EE30E70A71
:10673F0090067E747FF0A374FFF0900568E0FEA3CF
:10674F00E0FFC390067FE09FFF90067EE09EFEF085
:10675F00A3EFF0EE30E707E490067EF0A3F090068B
:09676F0099E0640260030267F581
:10677800856A57856B58C3E56294FFE561943F408D
:1067880027E5622401FFE56134C0FEEF2558F5587E
:10679800EE3557F557D3E55894FFE557947F401EDB
:1067A80075577F7558FF8016C374FF9562FF743F55
:1067B8009561FEC3E5589FF558E5579EF55775C393
:1067C8000E8551C28552C18553928554918555C213
:1067D8008556C190067EE0FEA3E0FF8E928F9175EC
:0B67E800C27F75C1FF85579285589154
:1067F300802D75C30E8551C28552C1855392855430
:10680300918555C28556C190067EE0FEA3E0FF8EBA
:10681300928F9175C27F75C1FF856192856291C226
:1068230081C281C28190067EE5CFF0A3E5CEF090D0
:10683300067EE030E707E490067EF0A3F090067E44
:07684300E0F568A3E0F56930
:01684A00222B
:106E6900AB69AA6875C3038AC28BC1759200759113
:106E790008C281C281859651859552E552640745BC
:106E8900517066F554755340EA540FFCEB54F07594
:106E9900C3038CC2F5C1759208759100C281C28184
:106EA900AC96AD95743C2DF58274603CF583E49302
:106EB9007A0075C3018AC2F5C1759200759140C205
:106EC90081C281AA94AB93EB4254EA42537A377B4D
:106ED9000075C3018553C28554C18A928B91C281C1
:106EE900C281AA96AB95026F8AE4F554E55225E072
:106EF900FFE55133FE74E32FF58274923EF58374F6
:106F09000193F553EA540FFCEB54F075C3038CC29B
:106F1900F5C1759208759100C281C281AC96AD9593
:106F2900743C2DF58274603CF583E4937A0075C353
:106F3900018AC2F5C1E55225E0FFE55133FE74E34C
:106F49002FF58274923EF583E493FE7401938E9239
:106F5900F591C281C281AA94AB93EB4254EA4253A0
:106F69007A377B0075C3018553C28554C18A928BD8
:106F790091C281C281AA96AB95EAA2E713FAEB13F3
:106F8900FB900699E014603E14603D2402703DAA0E
:036F990068AB6979
:106F9C0075C3038AC28BC18A928B91C281C28185CF
:106FAC00965585955675C3038555C28556C1759200
:106FBC0001759100C281C281AA96AB950BBB0001F1
:016FCC000ABA
:086FCD00800280008A5F8B60E6
:016FD5002299
:107C94009005C3E030E70F900621E0FFA3E09005D4
:107CA400B6CFF0A3EFF09005B6E0F551A3E0F5529E
:107CB400E42552F55274803551F551900633E0FEB7
:107CC400A3E07802CEC313CE13D8F9FF900572E077
:107CD400FAA3E0FBC3EF9BF554EE9AF553900686A6
:107CE400E030E12F75C30E8551C28552C185539290
:107CF40085549175C27F75C1FFE56EC313FEE56FB0
:107D0400138E92F5918570C28571C1855B92855CF5
:107D140091802175C30E8551C28552C185539285C8
:107D2400549175C27F75C1FFE56EC313FEE56F13F1
:107D34008E92F591C281C281C281ACCFADCEC3EC2B
:107D4400648094805003E4FCFD7466F551F552752B
:107D5400C3038CC28DC1855192855291C281C28167
:0F7D6400AC96AD9574992DFD74193CF5598D5A57
:017D730022ED
:0488F900AD07AC0615
:1088FD0090062BE0FEA3E07806CEC313CE13D8F975
:10890D002401FFEE34FE90067EF0A3EFF09006B347
:10891D00E0602D90067EE0FEA3E0FFD39400EE64B0
:10892D00809480400FEF2DFDEE3CFC30E7127C7FF4
:10893D007DFF800CEF2DFDEE3CFC30E703E4FCFDEC
:04894D00AE04AF05C0
:018951002203
:108183009005C3E030E60F900627E0FFA3E09005DB
:10819300B4CFF0A3EFF09005B4E0F551A3E0F552AE
:1081A300900631E0C313FEA3E013FF90056EE0FADF
:1081B300A3E0FBC3EF9BF554EE9AF553900686E0DC
:1081C30030E23575C30EE42552FFE5513480F5C224
:1081D3008FC185539285549175C27F75C1FFE56C3C
:1081E300C313FEE56D138E92F5918570C28571C13F
:1081F300855B92855C91802775C30EE42552FFE56C
:10820300513480F5C28FC185539285549175C27FD5
:1082130075C1FFE56CC313FEE56D138E92F591C234
:1082230081C281C281ACCFADCEC3EC648094805057
:0882330003E4FCFD8C728D7365
:01823B002220
:1069FF00E565147003026AC4147003026AE9147027
:106A0F0003026B0B147003026B3024D27003026B02
:106A1F004224326003026B4A9005C3E030E10F90CD
:106A2F000647E0FFA3E09005AACFF0A3EFF0900692
:106A3F0097E0605AE55E6432455D6034900546E04C
:106A4F00C313FEA3E013FF9006ACE02FFD9006AB3F
:106A5F00E03EFCE55E24CEFFE55D34FFFEEF7802FD
:106A6F00C333CE33CED8F92DF567EC3EF5668035BE
:106A7F009005AAE0C313FEA3E013FF9006ACE02F2E
:106A8F00F5679006ABE03EF566AF67FE80109005A8
:106A9F00AAE0C313F566A3E013F567FFAE6612888D
:106AAF00F98E668F67E56620E703026B4AE4F566A9
:106ABF00F567026B4A9005C3E030E30F900645E09F
:106ACF00FFA3E09005AECFF0A3EFF09005AEE0C3CB
:106ADF0013F561A3E013F56280619005C2E030E029
:106AEF000F900629E0FFA3E09005B8CFF0A3EFF0D9
:106AFF009005B8E0F56CA3E0F56D803F9005C2E01E
:106B0F0030E10F900623E0FFA3E09005BACFF0A38A
:106B1F00EFF09005BAE0C313F56EA3E013F56F80A5
:106B2F001AAF84E4F584D2EC90064DA3E0F59B8F69
:106B3F008480080574E5747002D21EE56530E10BA0
:106B4F0030E008127C94126CFB801DE56530E10883
:106B5F0012667F1274E88010E56530E005126E69E9
:106B6F008006124F6A1281830565E565D394324022
:046B7F0003E4F565D1
:016B830022EF
:1071CB0043061701062D43061A01063D41060D0025
:1071DB0041060E0041060F00410610004206110049
:0A71EB00024206150000C117C1188A
:10928400AF84E4F58475E881F5BBF5BA75BCA843F1
:04929400E7028F84DA
:0192980022B3
:1091FA00AF8475840275E888E4F5BAF5BB75BCC01E
:08920A0043BC0143E7108F840F
:019212002239
:0350300002760FF6
:10760F00C0E0C083C082C0D075D000C000C004C02D
:05761F0005C006C007D4
:10762400C2ED90060EE0FF25E0241DF582E4340649
:10763400F583E0FCA3E0FDC3E5BE9D90067BF0E589
:10764400BF9C90067AF0E0FCA3E0FDD39400EC64C8
:10765400809480404A90060DE0FEA807088002C38B
:1076640013D8FC30E00690060EE0805AD3ED9480E7
:10767400EC64809482500302771390060EE0FF2599
:10768400E0241DF582E43406F583E5BFF0A3E5BEEE
:10769400F07401A807088002C333D8FC4E806C90B4
:1076A400067AE0FEA3E0FFC3EE648094805060900D
:1076B400060EE0FD90060DE0FCA805088002C31349
:1076C400D8FC20E015ED25E0241DF582E43406F510
:1076D40083E5BFF0A3E5BEF08035C3EF9480EE648C
:1076E40080947D502A90060EE0FF25E0241DF5824B
:1076F400E43406F583E5BFF0A3E5BEF07401A80702
:10770400088002C333D8FCFFC3EC9F90060DF090B1
:0B771400060EE004F05407F0E0F5BBA7
:10771F00D007D006D005D004D000D0D0D082D083EF
:03772F00D0E03275
:03503900026B8483
:106B8400C0E0C0F0C083C082C0D075D000C000C0D7
:0D6B940001C002C003C004C005C006C00758
:106BA100C2EDAFBE8F488F49900617E0FBA3E0FA14
:106BB100A3E0F9900610E0FF75F002A4F58285F0DC
:106BC100831262D8FDACF0C3E5499D90067DF0E5E6
:106BD100489C90067CF0D3A3E0940090067CE0648E
:106BE100809480406990060FE0FEA807088002C3E8
:106BF10013D8FC30E014900617E0FBA3E0FAA3E001
:106C0100F9900610E075F0028074D390067DE0944F
:106C11006490067CE0648094805003026CD49006FA
:106C210017E0FBA3E0FAA3E0F9900610E0FF75F08E
:106C310002A4F58285F083E5488549F012632F743B
:106C410001A807088002C333D8FC4E026CD0C39060
:106C5100067CE064809480507A900610E0FF9006F4
:106C61000FE0FEA807088002C313D8FC20E01F90A4
:106C71000617E0FBA3E0FAA3E0F975F002EFA4F533
:106C81008285F083E5488549F012632F8045C390E2
:106C9100067DE0949C90067CE06480947F50349063
:106CA1000617E0FBA3E0FAA3E0F9900610E0FF75F8
:106CB100F002A4F58285F083E5488549F012632F3F
:106CC1007401A807088002C333D8FCFFC3EE9F906C
:0F6CD100060FF0900610E004F05407F0E0F5BB5A
:106CE000D007D006D005D004D003D002D001D00008
:0B6CF000D0D0D082D083D0F0D0E032B2
:0350150002460050
:10460000C0E0C0F0C083C082C0D075D000C000C080
:0D46100001C002C003C004C005C006C00701
:10461D00C2FF900611E0FEA3E0FF20E003024990E7
:10462D00AD9BA3E0F0A3E04DF0EF64034E7021E0ED
:10463D00C4F8540FC868FF900613E0C454F048F94D
:10464D0090061AE0FBA3E0FAA3E0C98FF012631005
:10465D00900611E0FEA3E0FF640F4E600302478C4D
:10466D00EF24FFFFEE34FFC313FEEF1324FEFFEE26
:10467D0034FFFEEF25E0FFEE33FE90061AE0FBA3BC
:10468D00E0FAA3E0F98F828E831262D8FFE5F0C4C1
:10469D00F854F0C868FEEFC4540F48FF900613E0BD
:1046AD00FCA3E0FDC39FFFEC9EFEA3F0A3EFF0D3B0
:1046BD009400EE64809480405C3017030247F8D379
:1046CD00900616E09403900615E0648094805003E4
:1046DD00024942900614E0C4F8540FC868FD9006D4
:1046ED0013E0C454F048FC900612E024FFFF90063E
:1046FD0011E034FFC313FEEF1324FEFFEE34FFFE73
:10470D00EF25E0FFEE338F82F583EC8DF012632FF2
:10471D00D217024942C3900615E06480948040038D
:10472D0002494220170302486AC3900616E094FD21
:10473D00900615E06480947F400302494290061470
:10474D00E0C4F8540FC868FD900613E0C454F04857
:10475D00FC900612E024FFFF900611E034FFC31316
:10476D00FEEF1324FEFFEE34FFFEEF25E0FFEE33E8
:10477D008F82F583EC8DF012632FC21702494290A0
:10478D000611E0FEA3E0FF640D4E60030248F9EF51
:10479D0024FFFFEE34FFC313FEEF1324FEFFEE34B0
:1047AD00FFFEEF25E0FFEE33FE90061AE0FBA3E0DF
:1047BD00FAA3E0F98F828E831262D8FFE5F0C4F878
:1047CD0054F0C868FEEFC4540F48FF900613E0FC88
:1047DD00A3E0FDC39FFFEC9EFEA3F0A3EFF0D394E7
:1047ED0000EE64809480406430180BEDC4F8540FD3
:1047FD00C868FDEC8076D3900616E09403900615FC
:10480D00E0648094805003024942900614E0C4F89D
:10481D00540FC868FD900613E0C454F048FC900690
:10482D0012E024FFFF900611E034FFC313FEEF13D7
:10483D0024FEFFEE34FFFEEF25E0FFEE338F82F511
:10484D0083EC8DF012632FD218024942C3900615E6
:10485D00E064809480400302494220183A90061487
:10486D00E0C4F8540FC868FD900613E0C454F04836
:10487D00FC900612E024FFFF900611E034FFC313F5
:10488D00FEEF1324FEFFEE34FFFEEF25E0FFEE33C7
:10489D008F82F58302493CC3900616E094FD900685
:1048AD0015E06480947F4003024942900614E0C4F1
:1048BD00F8540FC868FD900613E0C454F048FC90FE
:1048CD000612E024FFFF900611E034FFC313FEEF44
:1048DD001324FEFFEE34FFFEEF25E0FFEE338F8253
:1048ED00F583EC8DF012632FC2188049900614E009
:1048FD00C4F8540FC868FD900613E0C454F048FC8A
:10490D00900612E024FFFF900611E034FFC313FE62
:10491D00EF1324FEFFEE34FFFEEF25E0FFEE33FE36
:10492D0090061AE0FBA3E0FAA3E0F98F828E83ECE8
:10493D008DF012632F900611E475F0011262ACFE3A
:10494D00D3E5F09413EE94004014900611E4F0A317
:10495D007402F090064DE4F0A37484F0804D90063F
:10496D0012E024FEFF900611E034FFFEEF7802C343
:10497D0033CE33CED8F94484FF90064DEEF0A3EF3D
:10498D00F08028AF9B900613E4F0A3EFF0E0F8E47D
:10499D00F0E8900613F090064DE4F0A3F0900612A7
:0B49AD00E004F07006900611E004F03A
:1049B800D007D006D005D004D003D002D001D00053
:0B49C800D0D0D082D083D0F0D0E032FD
:1071F500C11B41069B004106A5FF48069C000000F7
:05720500000000000084
:10842C0090066BE5B0F0E4A3F090066CE0FFC3940B
:03843C0008507471
:10843F007401A807088002C333D8FCF52990066B96
:10844F00E0552924FF92089006A5E0FB55296030DE
:10845F0090069BE0FE552924FF920920083E200933
:10846F003BE5294EF0E529F4FFEB5F9006A5F09070
:0E847F00066CE0249CF582E43406F583E4F0FC
:10848D00801C3008099006A5E04529F08010900663
:0E849D006CE0249CF582E43406F583E004F0E4
:0884AB0090066CE004F08082F1
:0184B30022A6
:108B64007401A807088002C333D8FCFF90066DF097
:108B740090069BE0FE5F601090066DE0FF9006A5F6
:108B8400E05F60047F0180027F0090066EEFF0607A
:108B94000A90066DE0F45E90069BF090066EE0FF8E
:018BA40022AE
:028E2300AB079B
:108E25007401A807088002C333D8FC90066DF09042
:108E3500069BE0FE90066DE0FDF4FCEE5C90069B63
:108E4500F09006A5E04DF0749C2BF582E43406F510
:038E550083E4F0C3
:018E580022F7
:10917400749C2FF582E43406F583E0D3940840030D
:0B918400D38001C39209A209E433FF6D
:01918F0022BD
:0E92D40090066BE5B0F0E0540C1313543FFF0E
:0192E2002269
:0A933900AF84E4F58475D4978F84A7
:019343002207
:0A934400AF8475840175D4978F84FF
:01934E0022FC
:1086AC00AB84AAB1A2AF921C8F1A8E198D188C179D
:1086BC00AE19AF1A7878A60608A60753B10FE518BD
:1086CC00700543B110801BE51930E70543B13080CC
:1086DC001143B120431980AE19AF1A7878A6060859
:1086EC00A607E4F584C2AF43B701758F037878E62B
:1086FC00FE08E6F5828E83E4F053B7FEF58FA21CDC
:06870C0092AF8AB18B84DC
:018712002244
:10863700AB84AAB1A2AF921D8F108E0F8D0E8C0D39
:10864700AF0CEF3395E0FEEFF44E6050AE0FAF1076
:10865700787AA60608A60753B10FE50E700543B151
:1086670010801BE50F30E70543B130801143B1207F
:10867700430F80AE0FAF10787AA60608A607E4F579
:1086870084C2AF43B701758F01787AE6FE08E6F535
:10869700828E83E50CF053B7FEE4F58FA21D92AFEF
:0486A7008AB18B8485
:0186AB0022AC
:0E8B21008B2D8A2E892F8F338E328D318C3022
:108B2F00E4F536F537C3E5379535E53695345024FA
:108B3F0078301263721289A4AB2D052FE52FAA2E60
:108B4F007002052E14F9EF1262780537E53770D5EC
:048B5F00053680D186
:018B630022EF
:1089A400AB84AAB18F3B8E3A8D398C38AE3AAF3B4B
:1089B400787CA60608A60753B10FE539700543B1C4
:1089C40010801BE53A30E70543B130801143B120F4
:1089D400433A80AE3AAF3B787CA60608A607787C7B
:0F89E400E6FE08E6F5828E83E493FF8AB18B846A
:0189F3002261
:108AD9007D017F0412883B129157129299127F28C7
:108AE9001293391293441291FA12928475F70490F1
:108AF90006B7E0FF1292F143F6027FB87E2E12907C
:108B0900FE7F997E5712905C7FD77E0512907ED2A8
:088B1900AFE4F58475D10322DD
:10883B00AE8475840F758C20E4F58475EF06758412
:10884B000F758A83F59775840F758904F58475B751
:10885B003075840F4389018D8D758F018F8EFDFCD3
:10886B000DBD00010CE4B505F7ECB401F34389022F
:10887B00E58920E4120DEDAA0470010C14D39400C9
:0F888B00EA6480948140E9759702E4F58A8E844F
:01889A0022BB
:10915700AF8475840F75E10375E34075AD0175A59F
:0C9167000175A6BF75A04075A4E78F84B9
:0191730022D9
:10929900E4F584759A73759D1A43E60175F801C260
:0592A90087759B842283
:107F2800AE8475840F9006B4E07003027FBEC290E1
:107F3800752900752A10E52A152AAC297002152919
:087F4800D39400EC940050EE0C
:067F50007F28C286C285F5
:107F5600752900752A10E52A152AAC2970021529FB
:087F6600D39400EC940050EEEE
:027F6E00D285BA
:107F7000752900752A10E52A152AAC2970021529E1
:087F8000D39400EC940050EED4
:027F8800DFC850
:107F8A00752900752A10E52A152AAC2970021529C7
:087F9A00D39400EC940050EEBA
:027FA200D2907B
:107FA400752900752A10E52A152AAC2970021529AD
:0A7FB400D39400EC9400403C80ECF4
:067FBE007F28C286C28587
:107FC400752900752A10E52A152AAC29700215298D
:087FD400D39400EC940050EE80
:027FDC00D2854C
:107FDE00752900752A10E52A152AAC297002152973
:087FEE00D39400EC940050EE66
:047FF600DFC88E84CE
:017FFA002264
:1090FE00AD84E4F584F5C875C908C39FFFE49EF5F9
:0D910E00CB8FCA74FFF5CDF5CCD2CA8D848D
:01911B002231
:10905C00AD84758401E4F5C875C908C39FFFE49E0F
:10906C00F5CB8FCA74FFF5CDF5CC43E701D2CA8D91
:01907C00846F
:01907D0022D0
:10907E00AD84758402E4F5C875C908C39FFFE49EEC
:10908E00F5CB8FCA74FFF5CDF5CC43E704D2CA8D6C
:01909E00844D
:01909F0022AE
:10503C000000000300060009000C000F0012001510
:10504C000019001C001F002200250028002B002F37
:10505C00003200350038003B003E0041004500485E
:10506C00004B004E005100540057005A005E006186
:10507C0000640067006A006D007000730077007AAE
:10508C00007D0080008300860089008C008F0093D7
:10509C0000960099009C009F00A200A500A800AB00
:1050AC0000AE00B200B500B800BB00BE00C100C429
:1050BC0000C700CA00CD00D000D300D700DA00DD55
:1050CC0000E000E300E600E900EC00EF00F200F580
:1050DC0000F800FB00FE010101040107010A010DAB
:1050EC00011001140117011A011D012001230126D1
:1050FC000129012C012F013201350138013B013E00
:10510C000141014401470149014C014F0152015534
:10511C000158015B015E016101640167016A016D67
:10512C000170017301760179017C017E018101849A
:10513C000187018A018D0190019301960199019BD0
:10514C00019E01A101A401A701AA01AD01AF01B209
:10515C0001B501B801BB01BE01C001C301C601C943
:10516C0001CC01CE01D101D401D701DA01DC01DF80
:10517C0001E201E501E801EA01ED01F001F301F5BD
:10518C0001F801FB01FD0200020302060208020BFA
:10519C00020E0210021302160218021B021E02203B
:1051AC00022302260228022B022E02300233023680
:1051BC000238023B023D0240024302450248024AC9
:1051CC00024D024F025202550257025A025C025F14
:1051DC000261026402660269026B026E0270027363
:1051EC0002750278027A027D027F028102840286B5
:1051FC000289028B028E0290029202950297029A09
:10520C00029C029E02A102A302A502A802AA02AD60
:10521C0002AF02B102B302B602B802BA02BD02BFBB
:10522C0002C102C402C602C802CA02CD02CF02D118
:10523C0002D302D502D802DA02DC02DE02E002E37B
:10524C0002E502E702E902EB02ED02F002F202F4DF
:10525C0002F602F802FA02FC02FE03000302030447
:10526C0003070309030B030D030F031103130315AA
:10527C0003170319031B031D031F0321032203241C
:10528C0003260328032A032C032E03300332033492
:10529C00033603370339033B033D033F034103420A
:1052AC00034403460348034A034B034D034F035186
:1052BC0003530354035603580359035B035D035F05
:1052CC00036003620364036503670369036A036C89
:1052DC00036D036F03710372037403750377037813
:1052EC00037A037C037D037F03800382038303859E
:1052FC00038603880389038B038C038D038F039030
:10530C00039203930395039603970399039A039BC4
:10531C00039D039E039F03A103A203A303A503A65E
:10532C0003A703A803AA03AB03AC03AD03AF03B0FD
:10533C0003B103B203B303B503B603B703B803B9A0
:10534C0003BA03BC03BD03BE03BF03C003C103C246
:10535C0003C303C403C503C603C703C803C903CAF5
:10536C0003CB03CC03CD03CE03CF03D003D103D2A5
:10537C0003D303D403D503D603D703D703D803D958
:10538C0003DA03DB03DC03DC03DD03DE03DF03E012
:10539C0003E003E103E203E303E303E403E503E5D2
:1053AC0003E603E703E703E803E903E903EA03EB96
:1053BC0003EB03EC03ED03ED03EE03EE03EF03EF5E
:1053CC0003F003F003F103F103F203F203F303F32D
:1053DC0003F403F403F503F503F603F603F703F7FD
:1053EC0003F703F803F803F803F903F903F903FAD5
:1053FC0003FA03FA03FB03FB03FB03FB03FC03FCB1
:10540C0003FC03FC03FD03FD03FD03FD03FD03FE91
:10541C0003FE03FE03FE03FE03FE03FE03FF03FF76
:10542C0003FF03FF03FF03FF03FF03FF03FF03FF60
:10543C0003FF03FF03FF03FF03FF03FF03FF03FF50
:10544C0003FF03FF03FF03FE03FE03FE03FE03FE45
:10545C0003FE03FE03FD03FD03FD03FD03FD03FC3F
:10546C0003FC03FC03FC03FB03FB03FB03FB03FA3E
:10547C0003FA03FA03F903F903F903F803F803F841
:10548C0003F703F703F703F603F603F503F503F449
:10549C0003F403F303F303F203F203F103F103F058
:1054AC0003F003EF03EF03EE03EE03ED03ED03EC68
:1054BC0003EB03EB03EA03E903E903E803E703E780
:1054CC0003E603E503E503E403E303E303E203E19B
:1054DC0003E003E003DF03DE03DD03DC03DC03DBBB
:1054EC0003DA03D903D803D703D703D603D503D4E0
:1054FC0003D303D203D103D003CF03CE03CD03CC0C
:10550C0003CB03CA03C903C803C703C603C503C43B
:10551C0003C303C203C103C003BF03BE03BD03BC6B
:10552C0003BA03B903B803B703B603B503B303B2A5
:10553C0003B103B003AF03AD03AC03AB03AA03A8E1
:10554C0003A703A603A503A303A203A1039F039E22
:10555C00039D039B039A0399039703960395039367
:10556C0003920390038F038D038C038B03890388B1
:10557C0003860385038303820380037F037D037CFF
:10558C00037A037803770375037403720371036F53
:10559C00036D036C036A03690367036503640362A9
:1055AC000360035F035D035B035903580356035405
:1055BC0003530351034F034D034B034A0348034664
:1055CC00034403420341033F033D033B03390337C9
:1055DC000336033403320330032E032C032A03282F
:1055EC000326032403220321031F031D031B03199A
:1055FC000317031503130311030F030D030B030907
:10560C00030703040302030002FE02FC02FA02F881
:10561C0002F602F402F202F002ED02EB02E902E7FA
:10562C0002E502E302E002DE02DC02DA02D802D575
:10563C0002D302D102CF02CD02CA02C802C602C4F2
:10564C0002C102BF02BD02BA02B802B602B302B175
:10565C0002AF02AD02AA02A802A502A302A1029EF9
:10566C00029C029A0297029502920290028E028B81
:10567C000289028602840281027F027D027A02780C
:10568C00027502730270026E026B0269026602649A
:10569C000261025F025C025A025702550252024F2B
:1056AC00024D024A0248024502430240023D023BBF
:1056BC000238023602330230022E022B0228022656
:1056CC0002230220021E021B0218021602130210F1
:1056DC00020E020B020802060203020001FD01FB8E
:1056EC0001F801F501F301F001ED01EA01E801E532
:1056FC0001E201DF01DC01DA01D701D401D101CED5
:10570C0001CC01C901C601C301C001BE01BB01B876
:10571C0001B501B201AF01AD01AA01A701A401A11C
:10572C00019E019B0199019601930190018D018AC3
:10573C00018701840181017E017C0179017601736D
:10574C000170016D016A016701640161015E015B19
:10575C00015801550152014F014C014901470144C7
:10576C000141013E013B013801350132012F012C71
:10577C000129012601230120011D011A0117011421
:10578C000110010D010A01070104010100FE00FBDB
:10579C0000F800F500F200EF00EC00E900E600E391
:1057AC0000E000DD00DA00D700D300D000CD00CA45
:1057BC0000C700C400C100BE00BB00B800B500B2F9
:1057CC0000AE00AB00A800A500A2009F009C0099B1
:1057DC0000960093008F008C008900860083008067
:1057EC00007D007A007700730070006D006A00671E
:1057FC0000640061005E005A005700540051004ED6
:10580C00004B004800450041003E003B003800358D
:10581C000032002F002B002800250022001F001C46
:10582C00001900150012000F000C000900060003FF
:10583C000000FFFCFFF9FFF6FFF3FFF0FFEDFFEABE
:10584C00FFE6FFE3FFE0FFDDFFDAFFD7FFD4FFD079
:10585C00FFCDFFCAFFC7FFC4FFC1FFBEFFBAFFB732
:10586C00FFB4FFB1FFAEFFABFFA8FFA5FFA1FF9EEA
:10587C00FF9BFF98FF95FF92FF8FFF8CFF88FF85A2
:10588C00FF82FF7FFF7CFF79FF76FF73FF70FF6C59
:10589C00FF69FF66FF63FF60FF5DFF5AFF57FF5410
:1058AC00FF51FF4DFF4AFF47FF44FF41FF3EFF3BC7
:1058BC00FF38FF35FF32FF2FFF2CFF28FF25FF227B
:1058CC00FF1FFF1CFF19FF16FF13FF10FF0DFF0A30
:1058DC00FF07FF04FF01FEFEFEFBFEF8FEF5FEF2E5
:1058EC00FEEFFEEBFEE8FEE5FEE2FEDFFEDCFED99F
:1058FC00FED6FED3FED0FECDFECAFEC7FEC4FEC150
:10590C00FEBEFEBBFEB8FEB6FEB3FEB0FEADFEAAFA
:10591C00FEA7FEA4FEA1FE9EFE9BFE98FE95FE92A7
:10592C00FE8FFE8CFE89FE86FE83FE81FE7EFE7B54
:10593C00FE78FE75FE72FE6FFE6CFE69FE66FE64FE
:10594C00FE61FE5EFE5BFE58FE55FE52FE50FE4DA5
:10595C00FE4AFE47FE44FE41FE3FFE3CFE39FE364B
:10596C00FE33FE31FE2EFE2BFE28FE25FE23FE20EE
:10597C00FE1DFE1AFE17FE15FE12FE0FFE0CFE0A91
:10598C00FE07FE04FE02FDFFFDFCFDF9FDF7FDF434
:10599C00FDF1FDEFFDECFDE9FDE7FDE4FDE1FDDFD3
:1059AC00FDDCFDD9FDD7FDD4FDD1FDCFFDCCFDC96E
:1059BC00FDC7FDC4FDC2FDBFFDBCFDBAFDB7FDB505
:1059CC00FDB2FDB0FDADFDAAFDA8FDA5FDA3FDA09A
:1059DC00FD9EFD9BFD99FD96FD94FD91FD8FFD8C2B
:1059EC00FD8AFD87FD85FD82FD80FD7EFD7BFD79B9
:1059FC00FD76FD74FD71FD6FFD6DFD6AFD68FD6545
:105A0C00FD63FD61FD5EFD5CFD5AFD57FD55FD52CC
:105A1C00FD50FD4EFD4CFD49FD47FD45FD42FD4051
:105A2C00FD3EFD3BFD39FD37FD35FD32FD30FD2ED4
:105A3C00FD2CFD2AFD27FD25FD23FD21FD1FFD1C51
:105A4C00FD1AFD18FD16FD14FD12FD0FFD0DFD0BCD
:105A5C00FD09FD07FD05FD03FD01FCFFFCFDFCFB45
:105A6C00FCF8FCF6FCF4FCF2FCF0FCEEFCECFCEAC2
:105A7C00FCE8FCE6FCE4FCE2FCE0FCDEFCDDFCDB30
:105A8C00FCD9FCD7FCD5FCD3FCD1FCCFFCCDFCCB9A
:105A9C00FCC9FCC8FCC6FCC4FCC2FCC0FCBEFCBD02
:105AAC00FCBBFCB9FCB7FCB5FCB4FCB2FCB0FCAE66
:105ABC00FCACFCABFCA9FCA7FCA6FCA4FCA2FCA0C7
:105ACC00FC9FFC9DFC9BFC9AFC98FC96FC95FC9323
:105ADC00FC92FC90FC8EFC8DFC8BFC8AFC88FC8779
:105AEC00FC85FC83FC82FC80FC7FFC7DFC7CFC7ACE
:105AFC00FC79FC77FC76FC74FC73FC72FC70FC6F1C
:105B0C00FC6DFC6CFC6AFC69FC68FC66FC65FC6466
:105B1C00FC62FC61FC60FC5EFC5DFC5CFC5AFC59AC
:105B2C00FC58FC57FC55FC54FC53FC52FC50FC4FED
:105B3C00FC4EFC4DFC4CFC4AFC49FC48FC47FC462A
:105B4C00FC45FC43FC42FC41FC40FC3FFC3EFC3D64
:105B5C00FC3CFC3BFC3AFC39FC38FC37FC36FC3595
:105B6C00FC34FC33FC32FC31FC30FC2FFC2EFC2DC5
:105B7C00FC2CFC2BFC2AFC29FC28FC28FC27FC26F2
:105B8C00FC25FC24FC23FC23FC22FC21FC20FC1F18
:105B9C00FC1FFC1EFC1DFC1CFC1CFC1BFC1AFC1A38
:105BAC00FC19FC18FC18FC17FC16FC16FC15FC1454
:105BBC00FC14FC13FC12FC12FC11FC11FC10FC106C
:105BCC00FC0FFC0FFC0EFC0EFC0DFC0DFC0CFC0C7D
:105BDC00FC0BFC0BFC0AFC0AFC09FC09FC08FC088D
:105BEC00FC08FC07FC07FC07FC06FC06FC06FC0595
:105BFC00FC05FC05FC04FC04FC04FC04FC03FC0399
:105C0C00FC03FC03FC02FC02FC02FC02FC02FC0197
:105C1C00FC01FC01FC01FC01FC01FC01FC00FC0092
:105C2C00FC00FC00FC00FC00FC00FC00FC00FC0088
:105C3C00FC00FC00FC00FC00FC00FC00FC00FC0078
:105C4C00FC00FC00FC00FC01FC01FC01FC01FC0163
:105C5C00FC01FC01FC02FC02FC02FC02FC02FC0349
:105C6C00FC03FC03FC03FC04FC04FC04FC04FC052A
:105C7C00FC05FC05FC06FC06FC06FC07FC07FC0707
:105C8C00FC08FC08FC08FC09FC09FC0AFC0AFC0BDF
:105C9C00FC0BFC0CFC0CFC0DFC0DFC0EFC0EFC0FB0
:105CAC00FC0FFC10FC10FC11FC11FC12FC12FC1380
:105CBC00FC14FC14FC15FC16FC16FC17FC18FC1848
:105CCC00FC19FC1AFC1AFC1BFC1CFC1CFC1DFC1E0D
:105CDC00FC1FFC1FFC20FC21FC22FC23FC23FC24CD
:105CEC00FC25FC26FC27FC28FC28FC29FC2AFC2B88
:105CFC00FC2CFC2DFC2EFC2FFC30FC31FC32FC333C
:105D0C00FC34FC35FC36FC37FC38FC39FC3AFC3BEB
:105D1C00FC3CFC3DFC3EFC3FFC40FC41FC42FC439B
:105D2C00FC45FC46FC47FC48FC49FC4AFC4CFC4D41
:105D3C00FC4EFC4FFC50FC52FC53FC54FC55FC57E5
:105D4C00FC58FC59FC5AFC5CFC5DFC5EFC60FC6184
:105D5C00FC62FC64FC65FC66FC68FC69FC6AFC6C1F
:105D6C00FC6DFC6FFC70FC72FC73FC74FC76FC77B5
:105D7C00FC79FC7AFC7CFC7DFC7FFC80FC82FC8347
:105D8C00FC85FC87FC88FC8AFC8BFC8DFC8EFC90D3
:105D9C00FC92FC93FC95FC96FC98FC9AFC9BFC9D5D
:105DAC00FC9FFCA0FCA2FCA4FCA6FCA7FCA9FCABE1
:105DBC00FCACFCAEFCB0FCB2FCB4FCB5FCB7FCB962
:105DCC00FCBBFCBDFCBEFCC0FCC2FCC4FCC6FCC8DD
:105DDC00FCC9FCCBFCCDFCCFFCD1FCD3FCD5FCD757
:105DEC00FCD9FCDBFCDDFCDEFCE0FCE2FCE4FCE6CC
:105DFC00FCE8FCEAFCECFCEEFCF0FCF2FCF4FCF63F
:105E0C00FCF8FCFBFCFDFCFFFD01FD03FD05FD07A3
:105E1C00FD09FD0BFD0DFD0FFD12FD14FD16FD180A
:105E2C00FD1AFD1CFD1FFD21FD23FD25FD27FD2A6F
:105E3C00FD2CFD2EFD30FD32FD35FD37FD39FD3BD2
:105E4C00FD3EFD40FD42FD45FD47FD49FD4CFD4E2F
:105E5C00FD50FD52FD55FD57FD5AFD5CFD5EFD618B
:105E6C00FD63FD65FD68FD6AFD6DFD6FFD71FD74E3
:105E7C00FD76FD79FD7BFD7EFD80FD82FD85FD8738
:105E8C00FD8AFD8CFD8FFD91FD94FD96FD99FD9B8A
:105E9C00FD9EFDA0FDA3FDA5FDA8FDAAFDADFDB0D9
:105EAC00FDB2FDB5FDB7FDBAFDBCFDBFFDC2FDC425
:105EBC00FDC7FDC9FDCCFDCFFDD1FDD4FDD7FDD96E
:105ECC00FDDCFDDFFDE1FDE4FDE7FDE9FDECFDEFB3
:105EDC00FDF1FDF4FDF7FDF9FDFCFDFFFE02FE04F6
:105EEC00FE07FE0AFE0CFE0FFE12FE15FE17FE1A32
:105EFC00FE1DFE20FE23FE25FE28FE2BFE2EFE316F
:105F0C00FE33FE36FE39FE3CFE3FFE41FE44FE47AC
:105F1C00FE4AFE4DFE50FE52FE55FE58FE5BFE5EE6
:105F2C00FE61FE64FE66FE69FE6CFE6FFE72FE751F
:105F3C00FE78FE7BFE7EFE81FE83FE86FE89FE8C55
:105F4C00FE8FFE92FE95FE98FE9BFE9EFEA1FEA489
:105F5C00FEA7FEAAFEADFEB0FEB3FEB6FEB8FEBBBB
:105F6C00FEBEFEC1FEC4FEC7FECAFECDFED0FED3F1
:105F7C00FED6FED9FEDCFEDFFEE2FEE5FEE8FEEB21
:105F8C00FEEFFEF2FEF5FEF8FEFBFEFEFF01FF0447
:105F9C00FF07FF0AFF0DFF10FF13FF16FF19FF1C71
:105FAC00FF1FFF22FF25FF28FF2CFF2FFF32FF359D
:105FBC00FF38FF3BFF3EFF41FF44FF47FF4AFF4DC9
:105FCC00FF51FF54FF57FF5AFF5DFF60FF63FF66F1
:105FDC00FF69FF6CFF70FF73FF76FF79FF7CFF7F1B
:105FEC00FF82FF85FF88FF8CFF8FFF92FF95FF9844
:105FFC00FF9BFF9EFFA1FFA5FFA8FFABFFAEFFB16C
:10600C00FFB4FFB7FFBAFFBEFFC1FFC4FFC7FFCA93
:10601C00FFCDFFD0FFD4FFD7FFDAFFDDFFE0FFE3BA
:10602C00FFE6FFEAFFEDFFF0FFF3FFF6FFF9FFFCE1
:10603C000000010202030404050607070809090A07
:10604C000B0C0C0D0E0E0F1011111213141415163F
:10605C00171718191A1A1B1C1D1E1E1F202121226E
:10606C002324252526272829292A2B2C2D2D2E2F94
:10607C003031323233343536373738393A3B3C3DB0
:10608C003D3E3F40414243434445464748494A4BC5
:10609C004B4C4D4E4F5051525354555656575859D0
:1060AC005A5B5C5D5E5F60616263646566676869CC
:1060BC006A6B6C6C6D6E6F707172737475777879C6
:1060CC007A7B7C7D7E7F80818283848586878889AC
:1060DC008A8B8C8E8F9091929394959697989A9B8D
:1060EC009C9D9E9FA0A1A3A4A5A6A7A8A9ABACAD5F
:1060FC00AEAFB0B2B3B4B5B6B7B9BABBBCBDBFC026
:10610C00C1C2C4C5C6C7C8CACBCCCDCFD0D1D2D4DE
:10611C00D5D6D8D9DADBDDDEDFE1E2E3E5E6E7E888
:10612C00EAEBECEEEFF0F2F3F5F6F7F9FAFBFDFE25
:10720A00602005CB000000100080002000D0002084
:10721A0000E0002000B0002000C0001000D00020D4
:10722A0000E00030602005EB0000001000C00030D4
:10723A000080003000E0003000D0003000C00010B4
:10724A0000D0002000E00030C103011100C101C1DB
:10725A00024105C4000212000002140000011604D3
:02726A00C180E1
:0350120002500F3A
:03500F00C2CF32DB
:03502D0002911CD1
:09911C00C0E0C0D075D000C0070E
:0E912500C2CFAF111511EF7005D21B7511B638
:07913300D007D0D0D0E032DC
:035033000249D35C
:1049D300C0E0C0F0C083C082C0D075D000C000C0AA
:0D49E30001C002C003C004C005C006C0072B
:1049F00085B14AC2CF7584031269FF900698E0140E
:104A0000606224FE7003024AAF046003024ABCD213
:104A100000E51254E0FE7F0070047D0180027D00FD
:104A2000A20CE4335DFDE4B50708EEB4E0047F01B9
:104A300080027F00EF4D6019E51430E703D3800159
:104A4000C3920BA206B00B5008751200751300C27A
:104A50000CA20B9206D3E5139400E51294E0405C9F
:104A6000D20C8058E51220E7047F0180027F00A26B
:104A70000CE4335FFFE51230E7047E0180027E0024
:104A8000EE4F6018E51430E703D38001C3920BA208
:104A900006B00B5007A200B39200C20CA20B920604
:104AA000D3E5139400E51294E04011D20C800DD2AE
:104AB00000300508751200751300C205900699E0D4
:104AC000FD7008D51623751604800330000EE560CE
:104AD0002513F513E55F3512F512800DC3E5139527
:104AE00060F513E512955FF51290069AE0146041A7
:104AF0001460302402704DE51220E711E51325E023
:104B0000FFE51233FEEF2401F54CEE801EE5132580
:104B1000E0FFE51233FEC374FF9FF54C747F9EF5F2
:104B20004B8021E5132401F54CE5123480F54B80D0
:104B300013E51220E708754B7F754CFF8006754B17
:104B400080754C01854B70854C719006B4E06055C2
:104B5000E57030E704D2018002C201A201300201F7
:104B6000B3503E9006B9E054FCF0ED7005300119E9
:104B70008029900699E0B402269005AEE0FCA3E0FF
:104B8000FDD39400EC948140099006B9E04401F013
:104B9000800DC3EC947F50079006B9E04402F0D238
:104BA0000FA2019202758400634B80854BD3854C24
:104BB000D2758403E5642515F515E5633514F51400
:104BC000E515AE147805CEC313CE13D8F9F54C8E87
:104BD0004B25E0FFE54B33FE743C2FF58274503ECD
:104BE000F583E493F54B740193F54C75C303854B42
:104BF000C2854CC1855992855A91C281C2818596E0
:104C00004B85954CE4254CF54C7404354BF54B9095
:104C10000680E0FD7014E54CC4F8540FC868F54EEA
:104C2000E54BC454F048F54D8072EDC39405502413
:104C300053B10F90060BE042B19005C5A3E0FAA373
:104C4000E0F582E54C25E0FFE54B33FEE5822FF5EC
:104C500082EA803953B10F90060BE042B190063FD3
:104C6000E0FEA3E07802CEC313CE13D8F9FF90057F
:104C7000B3E02FFF9005B2E03E8F82F583E54C252F
:104C8000E0FFE54B33FEE5822FF582E5833EF583B9
:104C9000E493F54D740193F54E854AB1900681E099
:104CA000FD7014E54CC4F8540FC868F550E54BC4CA
:104CB00054F048F54F8072EDC39405502453B10F62
:104CC00090060CE042B19005C8A3E0FAA3E0F5829B
:104CD000E54C25E0FFE54B33FEE5822FF582EA80C7
:104CE0003953B10F90060CE042B190063DE0FEA3AF
:104CF000E07802CEC313CE13D8F9FF9005B1E02FB0
:104D0000FF9005B0E03E8F82F583E54C25E0FFE59E
:104D10004B33FEE5822FF582E5833EF583E493F580
:104D20004F740193F550854AB1E57230E70675720C
:104D300000757300C374FF9573F54C747F9572F51D
:104D40004B75C30E8572C28573C1854D92854E9198
:104D5000854BC2854CC1854F92855091C281C281DD
:104D6000C28185CF4B85CE4C634B80758401854BCA
:044D7000D3854CD2C9
:104D7400D007D006D005D004D003D002D001D00093
:0B4D8400D0D0D082D083D0F0D0E0323D
:02726C00C11E41
:104D8F00E49005C2F0A3F0900544E0FEA3E0FBAA77
:104D9F000690064BE0FEA3E0FFC3EF9BFFEE9AFEEB
:104DAF00E49400FDE49400FC900574126392900566
:104DBF0046E0FEA3E0FBAA06900647E0FEA3E0FF55
:104DCF00C3EF9BFFEE9AFEE49400FDE49400FC9089
:104DDF000578126392900548E0FEA3E0FBAA0690C7
:104DEF000649E0FEA3E0FFC3EF9BFFEE9AFEE494BB
:104DFF0000FDE49400FC90057C12639290054AE05C
:104E0F00FEA3E0FBAA06900645E0FEA3E0FFC3EF7A
:104E1F009BFFEE9AFEE49400FDE49400FC90058065
:104E2F0012639290054CE0FEA3E0FBAA0690061DCC
:104E3F00E0FEA3E0FFC3EF9BFFEE9AFEE49400FDBC
:104E4F00E49400FC90058412639290054EE0FEA35B
:104E5F00E0FBAA0690061FE0FEA3E0FFC3EF9BFF57
:104E6F00EE9AFEE49400FDE49400FC900588126332
:104E7F0092900550E0FEA3E0FBAA06900627E0FE05
:104E8F00A3E0FFC3EF9BFFEE9AFEE49400FDE494D2
:104E9F0000FC90058C126392900552E0FEA3E0FB9C
:104EAF00AA06900621E0FEA3E0FFC3EF9BFFEE9A58
:104EBF00FEE49400FDE49400FC9005901263929040
:104ECF000554E0FEA3E0FBAA06900629E0FEA3E04E
:104EDF00FFC3EF9BFFEE9AFEE49400FDE49400FC09
:104EEF00900594126392900556E0FEA3E0FBAA068C
:104EFF00900623E0FEA3E0FFC3EF9BFFEE9AFEE4D4
:104F0F009400FDE49400FC9005981263929005586C
:104F1F00E0FEA3E0FBAA06900639E0FEA3E0FFC384
:104F2F00EF9BFFEE9AFEE49400FDE49400FC9005E5
:104F3F009C12639290055AE0FEA3E0FBAA0690062E
:104F4F0037E0FEA3E0FFC3EF9BFFEE9AFEE4940071
:0B4F5F00FDE49400FC9005A0026392AA
:108CD500900546EEF0FDA3EFF09005AACDF0A3EDCB
:108CE500F0AB07AA06900647E0FEA3E0FFC3EF9BA3
:108CF500FFEE9AFEE49400FDE49400FC90057812E2
:0A8D050063929005C3E054FDF022D4
:108D0F00900558EEF0A3EFF09005BCEEF0A3EFF056
:108D1F00FBAA06900639E0FEA3E0FFC3EF9BFFEE30
:108D2F009AFEE49400FDE49400FC90059C1263927B
:088D3F009005C2E054FBF02294
:108D4700900554EEF0A3EFF09005B8EEF0A3EFF026
:108D5700FBAA06900629E0FEA3E0FFC3EF9BFFEE08
:108D67009AFEE49400FDE49400FC9005941263924B
:088D77009005C2E054FEF02259
:108D7F00900556EEF0A3EFF09005BAEEF0A3EFF0EA
:108D8F00FBAA06900623E0FEA3E0FFC3EF9BFFEED6
:108D9F009AFEE49400FDE49400FC9005981263920F
:088DAF009005C2E054FDF02222
:0463F0008F298D2A3A
:1063F400C20874017E00A807088005C333CE33CEDB
:10640400D8F990066CF0EE90066BF0201E2EE52A6B
:1064140025E0241DF582E43406F583E0FEA3E0FFC5
:10642400E52925E024A8F582E43405F583EEF0A3FC
:10643400EFF074FF9005C2F0A302650090066BE0D4
:10644400FEA3E0FF9005C2E05EFEA3E05F4E700392
:10645400026504E52925E02444F582E43405F58346
:10646400E0FEA3E0FBAA06E52A25E0241DF582E46C
:106474003406F583E0FEA3E0FFC3EF9BFFEE9AFE34
:10648400E49400FDE49400FC74FF7BC0FAF9F8D3B3
:1064940012635C5041E52925E02444F582E4340587
:1064A400F583E0FEA3E0FBAA06E52A25E0241DF51A
:1064B40082E43406F583E0FEA3E0FFC3EF9BFFEE26
:1064C4009AFEE49400FDE49400FCE47B40FAF9F8BD
:1064D400C312635C5003128DEDE52A25E0241DF5FB
:1064E40082E43406F583E0FEA3E0FFE52925E024F9
:1064F400A8F582E43405F583EEF0A3EFF07F0022E3
:10650400E52925E02444F582E43405F583E0FEA37F
:10651400E0FBAA06E52A25E0241DF582E43406F50D
:1065240083E0FEA3E0FFC3EF9BFFEE9AFEE494003A
:10653400FDE49400FC90066D126392E52925E025A4
:10654400E02474F582E43405F583E0FCA3E0FDA3C4
:10655400E0FEA3E0FF900671126392E529B40112F4
:10656400900697E0600CE55E6432455D6004C20805
:10657400804A900671E0FCEC33401DE4FFFEFDFC14
:1065840090066DE0F8A3E0F9A3E0FAA3E0FBD312D0
:10659400635C5004D2088024E4FFFEFDFC90067185
:1065A400E0F8A3E0F9A3E0FAA3E0FBD312635C50A4
:1065B4000B90066DE0FCEC334002D2082008030285
:1065C400665590066BE0FEA3E0FF9005C2E04EF036
:1065D400A3E04FF0E52A25E0241DF582E43406F516
:1065E40083E0FEA3E0FFE52925E02444F582E434BA
:1065F40005F583EEF0A3EFF0E52A25E0241DF582EE
:10660400E43406F583E0FEA3E0FFE52925E024A8B1
:10661400F582E43405F583EEF0A3EFF0E47F40FE69
:10662400FDFC900671E0F8A3E0F9A3E0FAA3E0FB17
:10663400D312635C501674FF7FC0FEFDFC9006719C
:10664400E0F8A3A3A3E0C312635C5029128DED808C
:1066540024E52925E02444F582E43405F583E0FEAD
:10666400A3E0FFE52925E024A8F582E43405F583B9
:0A667400EEF0A3EFF0A208E433FFFC
:01667E0022F9
:0493970006040200C6
:0E726E004506B90000000000C11F4106B8002F
:108BE500E4F52A530707EF540390939793FEEFC3D9
:108BF500940450159006BDE0FFEDA806088002C359
:108C050033D8FC4F9006BDF0229006BCE0FFEDA8DE
:0D8C150006088002C333D8FC4F9006BCF067
:018C2200222F
:1091C7009006B9E0FE5306F3EF60047F0880027F44
:0991D70004EF42069006B9EEF027
:0191E000226C
:107FFB00900680E0D3940440047F0180027F008FC1
:10800B0029900681E0D3940440047F0180027F0015
:10801B00AC07E49006BCF0A3F0900680E0900564FA
:10802B00F025E025E024CBF582E43405F583A3E0CD
:10803B00FAA3E0FFEA4480FAA9079005C5E4F0A390
:10804B00EAF0A3E9F0900680E0FF25E025E024CEDE
:10805B00F582E43405F583E090060BF07D01128B7D
:10806B00E5900681E0FF900563F00D128BE590061D
:10807B0081E0FF25E025E024EBF582E43405F58370
:10808B00A3E0FAA3E0FBEA4480FAA9039005C8E455
:10809B00F0A3EAF0A3E9F0EF25E025E024EEF5826A
:1080AB00E43405F583E090060CF09006B4E060072D
:0780BB00AF04AD291291ACE6
:0180C200229B
:0B934F00900696E0FF1291C7027FFB22
:10839500C208E490066BF0A3F07F06129174EF60BB
:1083A500267F06128E23201F1A900696E070047F02
:1083B5000180027F00900696EFF0900562F0129121
:1083C500C7D208D21F80267F06128B64EF601E304D
:1083D5001F04C21F8017900696E0700590068080E6
:1083E50003900681E004F0E05407F0D208127FFB09
:1083F5009006B4E0602B900681E0C394054006909A
:10840500066C7401F0900680E0C394054006900662
:108415006B7401F090066CE0FF90066BE0FD129125
:06842500ACA208E433FFE5
:01842B00222E
:1085B900AC079006BBE05430F0ED603A9006B4E0A9
:1085C9006002800EEC14601214601714601A240300
:1085D900705B9006BBE04402F0229006BBE04408C1
:1085E900F0229006BBE0800A9006BBE04402F0440A
:1085F90008F04480F0229006B4E07031EC14601267
:1086090014601714601A240370239006BBE0440118
:10861900F0229006BBE04404F0229006BBE0800AF9
:0E8629009006BBE04401F04404F04440F0220F
:1091AC00AE079006BBE054CFF0EE6004E04410F044
:0B91BC00ED60079006BBE04420F022AD
:108F27009006B9E0548FF0EF14600F146014240218
:108F370070179006B9E04440F0229006B9E044204B
:0A8F4700F0229006B9E04410F02279
:108F7A00AD079006BAE054E3F0ED30E004E04410A7
:108F8A00F0ED30E1079006BAE04408F0ED30E20770
:088F9A009006BAE04404F02245
:108EC200AD079006BAE054FCF09006B9E0547FF08A
:108ED200ED14600F146014240270179006B9E04478
:108EE20080F0229006BAE04401F0229006BAE044F3
:038EF20002F02269
:108FA200AD079006BAE0541FF0ED30E004E04480D3
:108FB200F0ED30E1079006BAE04440F0ED30E20710
:088FC2009006BAE04420F02201
:1090A000EF14601214601314600824037011E4FFBD
:1090B000800A7F0480067F0180027F02128FA22235
:108E590090066BE572F0A3E573F090066BE090065F
:108E69006DF0E0FFC374FF9FF0E0C313FFF09006BD
:108E7900B8E06F600F90066DE0FF9006B8F053A060
:048E8900C0EF42A054
:018E8D0022C2
:10901500EF540314600F146014240270179006B9FE
:10902500E054FCF0229006B9E04402F0229006B923
:05903500E04401F022FF
:107D7400900677E584F075840F9006B4E0601AC22B
:017D8400906E
:107D8500752B00752C10E52C152CAE2B7002152BC0
:087D9500D39400EE940050EEBF
:107D9D00E4900675F0900675E0FFC394054003026C
:027DAD007E2C2A
:107DAF0074B92FF582E43406F583E0F52BE49006E1
:0C7DBF0076F0900676E0FFC39408505860
:107DCB0074017E00A807088005C333CE33CED8F9E3
:0E7DDB00FFEF552B24FF9209A2099286C28564
:107DE900752C00752D10E52D152DAE2C7002152C56
:087DF900D39400EE940050EE5B
:027E0100D28528
:107E0300752C00752D10E52D152DAE2C7002152C3B
:087E1300D39400EE940050EE40
:087E1B00900676E004F0809E61
:0F7E2300900675E004F0027DA29006B4E0601AAC
:107E3200752B00752C10E52C152CAE2B7002152B12
:087E4200D39400EE940050EE11
:087E4A00D290900677E0F58468
:017E5200220D
:1089F4009006B4E06008D290E4FDFF1291AC9006BA
:108A0400A4E0FF900697E0FD1285B9900698E0FF78
:108A14001290A0900686E0FF128F7A90069AE0FFEB
:108A2400128F27E4FF129015900686E0FF128F7ACA
:0E8A3400900699E0FF128EC212934F027D74DD
:10922B00000002AB055508000AAB0D55100012AB40
:08923B00155518001AAB1D5572
:02727C00C11A35
:02796B00A9076A
:10796D00E975F00C84ABF07A00E975F00C8424FF16
:10797D00F533E434FFF532EA6003027A1DEBB40C03
:10798D00004003027A1D90799AF82828730279BE77
:10799D000279C40279CA0279D00279D60279DC0261
:1079AD0079E20279E80279EE0279F4027A01027A3B
:1079BD000F7A007B03805D7A007B0480577A007B11
:1079CD000580517A007B06804B7A007B0780457AD3
:1079DD00007B08803F7A007B0980397A007B0A8022
:1079ED00337A007B0B802DE4FAFB0533E5337024ED
:1079FD00053280207A007B010533E53370160532A0
:107A0D0080127A007B020533E5337008053280045D
:107A1D00E4FEFF22E533C43354E0FEE4F5318E304D
:107A2D00F52FF52EEB25E0FFEA33FE742B2FF582B3
:107A3D0074923EF583E493FE740193FFE4FCFDE53F
:107A4D00312FF531E5303EF530ED352FF52FEC3595
:107A5D002EF52EE9D394674009E47531FF7530FF9B
:107A6D00800BE9C394095009E4F531F530F52FF594
:057A7D002EAE30AF3118
:017A820022E1
:107A83008D1BEF14604A24ECB40B004003027B8B84
:107A9300907AA175F003A4C58325F0C58373027A98
:107AA300C2027B8B027AE5027AF6027AF9027B162E
:107AB300027B33027B3E027B51027B64027B77E5D0
:107AC3001B75F00A84FF900698F01290A07F0122A4
:0F7AD300E51B25E0F51BF51CAF1DAE1C128D0F3A
:107AE2007F0122E51B75F00A84FF900686F0128F53
:107AF2007A7F01227F0022E51B75F00A84900699A5
:107B0200F0D3940240037402F0900699E0FF128EC3
:107B1200C27F0122E51B75F00A8490069AF0D39485
:107B22000240037402F090069AE0FF128F277F0151
:107B320022E51B75F00A849006818009E51B75F029
:107B42000A84900680F05407F0127FFB7F0122E541
:107B52001B25E0F51B751B00AF1B7E00128D477FB6
:107B62000122E51B25E0F51B751B00AF1B7E0012F1
:107B72008D7F7F0122E51BFD7C0075F004A4AEF031
:0F7B82002DF55EEC3EF55D80037F00227F002233
:067B91008B298A2A892BD2
:107B970090000312624B90066BF0E0FD540FA3F0C8
:107BA700FC9006A4E0FF74017E00A807088005C3C7
:107BB70033CE33CED8F9FFECFBEF5B24FF9208ED11
:107BC70054F02450603424D0606424F07003027CA5
:0E7BD7009124606003027C91200803027C91DF
:107BE500AB29AA2AA92B90000512624BFF12796BCB
:097BF5008E2C8F2D128CD5D205C7
:107BFE00027C91200803027C91AB29AA2AA92B9022
:107C0E00000512624B641F707A90000612624B756B
:107C1E005D00F55ED39433E55D94004066E55E1538
:107C2E005E7060155D805C300859AB29AA2AA92BBD
:107C3E0090000612624B25E09006A8F0A3E4F090A7
:107C4E00000512624B75F004A4FF9006A8E045F003
:107C5E00FEA3E04FFF9006A8EEF0A3EFF02401FF85
:107C6E00EE34809006ABF0A3EFF09006ABE0FEA3EF
:107C7E00E07803CEA2E713CE13D8F8F0EE9006AB61
:057C8E00F080007F0002
:017C930022CE
:108BA500AB84A2AF9209E4FDED8F3F8E3EF53DF516
:108BB5003CAE3EAF3F787CA60608A607F584C2AF5B
:108BC50043B701438F02438F0118E6FE08E6F5829D
:0F8BD5008E83E4F053B7FEF58FA20992AF8B8425
:018BE400226E
:028A4200AB0582
:108A4400AA84A2AF9209E4FDED8F458E44F543F567
:108A540042EBFF3395E0FEEFF44E6027AE44AF45A2
:108A6400787CA60608A607E4F584C2AF43B701756F
:108A74008F0118E6FE08E6F5828E83EBF053B7FE0D
:098A8400E4F58FA20992AF8A8487
:018A8D0022C6
:108C23008E3C8F3D8C3E8D3F8A408B41E5414540D4
:108C33006029853F82853E83E0FDAF3DAE3C128ACD
:108C430042E541154170021540053FE53F700205BD
:0C8C53003E053DE53D70D5053C80D1227A
:06939100E4F51EF51F22A9
:10919000AF1FAE1E128BA57C007D007B007A04AF52
:0C91A0001FAE1E128C23E4F51EF51F22EA
:06853A008E388F39A905FF
:10854000EE54FCFEE51F7003EE651E6059E51F4505
:108550001E6003129190E53854FCF51E751F00F55E
:108560003A851F3B7E007F009006737404F0A3E4FD
:10857000F0053BE53BAC3A7002053A14F5828C837A
:10858000E493FD0FEFAA0670010E14F5828A83EDC5
:10859000F0900674E024FFF0900673E034FFF0E002
:1085A0007002A3E070CBE5385403FE74002539F562
:0885B0008274003EF583E9F03E
:0185B80022A0
:108C9A008E318F328B338A348935E5371537AE36C4
:108CAA00700215364E60230532E532AE3170020588
:108CBA003114FFAB330535E535AA34700205341497
:0B8CCA00F9126232FD12853A80D022C0
:03000000024000BB
:03000300025003A5
:03000B000250069A
:030013000250098F
:03001B0002500C84
:0300230002500F79
:03002B000250126E
:0300330002501563
:03003B0002501858
:0300430002501B4D
:03004B0002501E42
:0300530002502137
:03005B000250242C
:0300630002502721
:03006B0002502A16
:0300730002502D0B
:03007B0002503000
:03008300025033F5
:03008B00025036EA
:03009300025039DF
:03009B0002503CD4
:0300A30002503FC9
:10400000787FE4F6D8FD9000007F007E20E4F0A3E6
:0A401000DFFCDEFA75817D024055E9
:10401A0002409AE493A3F8E493A34003F68001F2E2
:10402A0008DFF48029E493A3F85407240CC8C333A7
:10403A00C4540F4420C8834004F456800146F6DF76
:10404A00E4800B0102040810204080907136E47E5F
:10405A00019360BCA3FF543F30E509541FFEE4936B
:10406A00A360010ECF54C025E060A840B8E493A332
:10407A00FAE493A3F8E493A3C8C582C8CAC583CA5D
:10408A00F0A3C8C582C8CAC583CADFE9DEE780BE15
:01727E00000F
:10613C00E709F608DFFA8046E709F208DFFA803E45
:10614C0088828C83E709F0A3DFFA8032E309F60832
:10615C00DFFA8078E309F208DFFA807088828C839A
:10616C00E309F0A3DFFA806489828A83E0A3F6084E
:10617C00DFFA805889828A83E0A3F208DFFA804C28
:10618C0080D280FA80C680D4806980F280338010FF
:10619C0080A680EA809A80A880DA80E280CA803368
:1061AC0089828A83ECFAE493A3C8C582C8CCC583E0
:1061BC00CCF0A3C8C582C8CCC583CCDFE9DEE780B0
:1061CC000D89828A83E493A3F608DFF9ECFAA9F02F
:1061DC00EDFB2289828A83ECFAE0A3C8C582C8CC85
:1061EC00C583CCF0A3C8C582C8CCC583CCDFEADE9E
:1061FC00E880DB89828A83E493A3F208DFF980CC00
:10620C0088F0EF60010E4E60C388F0ED2402B404F8
:10621C000050B9F582EB2402B4040050AF2323459F
:06622C00822390618C73D7
:10623200BB010689828A83E0225002E722BBFE026A
:09624200E32289828A83E493229D
:10624B00BB010CE58229F582E5833AF583E0225008
:10625B0006E92582F8E622BBFE06E92582F8E22252
:0D626B00E58229F582E5833AF583E493226C
:10627800BB010689828A83F0225002F722BBFE0105
:02628800F322FF
:10628A00F8BB010DE58229F582E5833AF583E8F04A
:10629A00225006E92582C8F622BBFE05E92582C8F6
:0262AA00F222DE
:1062AC00C5F0F8A3E028F0C5F0F8E582158270027D
:0662BC001583E038F0221A
:1062C200A3F8E0C5F025F0F0E5821582700215838F
:0662D200E0C838F0E822EC
:1062D800BB0110E58229F582E5833AF583E0F5F004
:1062E800A3E0225009E92582F886F008E622BBFEE1
:1062F8000AE92582F8E2F5F008E222E5832AF58327
:08630800E993F5F0A3E99322EB
:10631000BB010A89828A83F0E5F0A3F0225006F7D8
:0F63200009A7F01922BBFE06F3E5F009F31922D5
:10632F00F8BB0111E58229F582E5833AF583E8F0A0
:10633F00E5F0A3F0225009E92582C8F608A6F0225D
:0D634F00BBFE09E92582C8F2E5F008F22244
:10635C00EB9FF5F0EA9E42F0E99D42F0EC6480C8B8
:06636C0064809845F02258
:106372007401FF3395E0FEFDFC080808E6CF2FF616
:1063820018E6CE3EF618E6CD3DF618E6CC3CF622EF
:0C639200ECF0A3EDF0A3EEF0A3EFF0227E
:10639E00D083D082F8E4937012740193700DA3A38E
:1063AE0093F8740193F5828883E4737402936860A2
:0663BE00EFA3A3A380DFA2
:1063C400EF4E6012EF60010EEDBB010B89828A83F0
:1063D400F0A3DFFCDEFA2289F05007F709DFFCA9FD
:0C63E400F022BBFEFCF309DFFCA9F02254
:00000001FF
